:020000040001F9
:10900000E0220020F9920100019301000393010086
:10901000059301000793010009930100000000007F
:109020000000000000000000000000000B930100A1
:109030000D930100000000000F9301001193010047
:109040006196010013930100D1990100139301006F
:109050001393010000000000999401001393010094
:109060001393010013930100139301001393010064
:109070001393010013930100139301001393010054
:1090800013930100B996010013930100139301009B
:10909000DD96010013930100E19601001393010096
:1090A0001393010013930100000000000000000072
:1090B0001393010013930100000000000000000062
:1090C00000000000000000000000000000000000A0
:1090D0000000000000000000000000000000000090
:1090E0000000000000000000000000000000000080
:1090F0000000000000000000000000000000000070
:10910000000000000000000000000000000000005F
:10911000000000000000000000000000000000004F
:10912000000000000000000000000000000000003F
:10913000000000000000000000000000000000002F
:10914000000000000000000000000000000000001F
:10915000000000000000000000000000000000000F
:1091600000000000000000000000000000000000FF
:1091700000000000000000000000000000000000EF
:1091800000000000000000000000000000000000DF
:1091900000000000000000000000000000000000CF
:1091A00000000000000000000000000000000000BF
:1091B00000000000000000000000000000000000AF
:1091C000000000000000000000000000000000009F
:1091D000000000000000000000000000000000008F
:1091E000000000000000000000000000000000007F
:1091F000000000000000000000000000000000006F
:10920000DFF80CD000F00AF9004800479DAB0100E0
:10921000E022002030B4044654E8000F0D4644E834
:109220000053002BF8D1156030BC704730B40446B1
:1092300054E8000F40EA010544E80053002BF7D141
:10924000156030BC704730B4044654E8000F00EAA3
:10925000010544E80053002BF7D1156030BC70477E
:1092600030B4044654E8000F80EA010544E8005396
:10927000002BF7D1156030BC704730B4044654E879
:10928000000F00EB010544E80053002BF7D11560F7
:1092900030BC704730B4044654E8000FA0EB010521
:1092A00044E80053002BF7D1156030BC704770B410
:1092B00004464FF0000054E8006F0D68AE4207BF4F
:1092C00044E80023012044E800630E60002B1CBF2B
:1092D0000020F0E770BC704730B4044654E8000F3B
:1092E00088422CBF451A054644E80053002BF5D1AF
:1092F000156030BC704700000648804706480047AC
:10930000FEE7FEE7FEE7FEE7FEE7FEE7FEE7FEE735
:10931000FEE7FEE7E5960100019201002DE9F05F0E
:109320000546002092469B468846064681464024D4
:109330001BE0284641464746224600F05EF8534669
:109340005A46C01A914110D311461846224600F0E1
:1093500016F82D1A67EB01084F462246012000211E
:1093600000F00DF817EB00094E41201EA4F1010496
:10937000DFDC484631462A464346BDE8F09F202AB6
:1093800004DB203A00FA02F1002070479140C2F15C
:10939000200320FA03F319439040704700487047B8
:1093A000D8CE010040EA01039B0703D009E008C9B9
:1093B000121F08C0042AFAD203E011F8013B00F89A
:1093C000013B521EF9D27047D2B201E000F8012BE6
:1093D000491EFBD270470022F6E710B513460A4635
:1093E00004461946FFF7F0FF204610BD421C10F856
:1093F000011B0029FBD1801A7047202A04DB203A88
:1094000021FA02F00021704721FA02F3D040C2F1A4
:10941000200291400843194670470000064C074D52
:1094200006E0E06840F0010394E807009847103434
:10943000AC42F6D3FFF7E8FE20D5010040D501008D
:1094400070B58C1810F8015B15F0070301D110F806
:10945000013B2A1106D110F8012B03E010F8016B33
:1094600001F8016B5B1EF9D12B0705D40023521EB6
:109470000DD401F8013BFAE710F8013BCB1A921C1E
:1094800003E013F8015B01F8015B521EF9D5A1421C
:10949000D8D3002070BD00002DE9F04700268AB027
:1094A000DFF85091B0464FF4807501243746069698
:1094B000284601F021FF38B1D9F80403204203D037
:1094C000284601F00FFF26432D1D64007F1CADB21E
:1094D000082FEDD34FF4BE74204601F00DFF48B1C4
:1094E000204601F0FFFE46F0004606AA01210020BA
:1094F00001F0E4FE404D16F0FF0F15D001270024C7
:1095000037420DD009EB8401D1F81005D1F81015C0
:10951000C0F3042055F82420C1F3014102B1904763
:109520007F00641C082CEBD3002E5FDA4FF0FF3075
:10953000CDF8108054E0281910F8507F90F9000001
:1095400027F0C008401C3BD007A9404601F0CCFCE6
:1095500010B34FEA9719404600F0FEFF55F820700F
:109560001FB1B9F1030F03D006E0B9F1030F27D102
:1095700004A9404601F0C0FC4FF0A04101EB880077
:10958000D0F8000706A9C0F3014A404601F0ACFC40
:1095900018B1BAF1020F03D012E0BAF1030F0FD1E4
:1095A000B9F1030F08D1BAF1020F1DD002214046D4
:1095B00001F068FE761CF6B217B149464046B8473E
:1095C000641C042CB7D3002E10D06A460121002061
:1095D00001F074FE06990098884207D0069004981E
:1095E000002634460790A6E70321E0E70AB0BDE86D
:1095F000F087000000600040F413002000F01F021C
:10960000012191404009800000F1E020C0F8801263
:10961000704700F01F02012191404009800000F1D5
:10962000E020C0F80011704700F01F0201219140B6
:109630004009800000F1E020C0F80012704749079F
:10964000090E002806DA00F00F0000F1E02080F893
:10965000141D704700F1E02080F8001470470000EE
:1096600070B54FF48076304601F050FC114CB505D2
:1096700060B1304601F051FC0120C5F80803607963
:1096800020B9012060712168002088474FF482765C
:10969000304601F03BFC00280AD0304601F03DFC8A
:1096A0000220C5F808032168BDE870400120084782
:1096B00070BD00005412002007480021C0F840117E
:1096C000C0F84411C0F84811C0F84C11C0F800119E
:1096D000C0F8041103F09EB80010014002F0E8BF8A
:1096E00002F02CBBF0B5A848A74B012600781B1D43
:1096F0001A1D4FF0805106280BD11C78240708D181
:109700001478C4F30314032C06D0042C04D0052CC5
:1097100002D0062807D011E0B1F824439B4DC4F3D2
:1097200004242C6002E01C78240707D11478C4F3C9
:109730000314032C02D1974D954C6C67D1F830512E
:10974000D1F84442944FC4F342343C6006280CD113
:109750001C78240709D11478C4F30314032C04D112
:109760008E4C276827F0807727604FF080470024D1
:10977000C7F80C41C7F81041874F3F1F3C600628CF
:1097800007D11F783F0704D11778C7F30317032FBA
:1097900002D0062808D01FE0DFF8FCC103270CF137
:1097A000640CCCF8007007E01F783F0714D11778DD
:1097B000C7F30317032F0FD1DFF8E4C10527CCF857
:1097C0000070774F78373E60754F08373C600CF17A
:1097D000040C3F27CCF80070724F3F68DFF8C8C117
:1097E000CCF800706F4F3F1D3F680CF1040CCCF8B3
:1097F00000706C4F08373F680CF1040CCCF8007017
:10980000684F0C373F680CF1040CCCF80070654FC2
:1098100010373F680CF1040CCCF80070614F14371E
:109820003F680CF1040CCCF800705E4F18373F68AD
:10983000DFF874C10CF1200CCCF80070594F1C37C4
:109840003F680CF1040CCCF80070564F20373F688D
:109850000CF1040CCCF80070524F24373F680CF127
:10986000040CCCF800704F4F28373F680CF1040C03
:10987000CCF800704B4F2C373F680CF1040CCCF83F
:109880000070484F30373F68DFF81CC10CF1400CC6
:10989000CCF80070434F34373F680CF1040CCCF81F
:1098A0000070404F38373F680CF1040CCCF8007062
:1098B0003C4F3C373F680CF1040CCCF80070394F3A
:1098C00040373F680CF1040CCCF80070DFF8DCC0C6
:1098D000FB27CCF80070062813D11F783F0710D162
:1098E0001778C7F30317032F03D0042F01D0052FD8
:1098F00007D1D1F85872DFF8B8C007F04F07CCF89D
:1099000000702C480268D20702D06FF0010202609A
:10991000062D08D1D1F83401062804D12648016863
:1099200041F4806101604FF01021D1F8000200285D
:1099300003DBD1F80402002822DA204A166020480E
:109940000368002BFCD01523C1F800320568002DF8
:10995000FCD0C1F8043201680029FCD01460016811
:109960000029FCD0BFF34F8F0C48F0380168154A2E
:1099700001F4E06111430160BFF34F8F00BFFDE7C9
:10998000124911480860F0BDE00F00F04035014079
:109990000DF0ADBA00C007403C050040FCED00E012
:1099A000105600400404001020C5004018F5004087
:1099B000E40E0040000400403C17004004E5014074
:1099C00000E401400400FA050090D0030C130020CD
:1099D0000149024802F09EBF5014002000200040C0
:1099E00002E008C8121F08C1002AFAD17047704768
:1099F000002001E001C1121F002AFBD170470000C6
:109A00000121202803DA81400548014003E0402875
:109A100002DA2038814009B10120704700207047E8
:109A2000FC06FFBD082806D228B1012803D004286F
:109A300001D00120704700207047000030B593B07E
:109A40005920ADF83C00184811901720ADF840009F
:109A500004253C216846FFF7BEFC00240FA88DF8C2
:109A6000004009908DF8035018211048FFF7B3FC0F
:109A70000E4805210C4A017044600475A0218160E4
:109A80008481103A684602CA00F0C0F908B100F0BB
:109A90009FF80549054A1039081F72DF002801D0D8
:109AA00000F096F813B030BD241200203C130020C3
:109AB000022000F0C7BA000070B50024064D06E091
:109AC0006868012110F8340002F004FA641C287858
:109AD0008442F5D3002070BD60120020F8B5154611
:109AE0000C460646052A01D20720F8BD02F0EEFA20
:109AF00018B902F0B3FA0028F7D1124900224E60DB
:109B00000C708D60C1E90422C1E906220E4D0DE002
:109B100006EBC4002968009181788DF80110007867
:109B20000A4A694602F028FA0028DED1641EE4B22F
:109B3000EED2BDE8F84004480021054A001D00F0BF
:109B400053B800006012002004CC0100CDA7010032
:109B5000E1A6010072B601F063FE00BF01F0A2FCB5
:109B60000028FBD1104C0121208801EB00400FA1FF
:109B700001F0A8FD10480068C00700D000BE208892
:109B8000022101EB00400DA101F09CFDBFF34F8FBE
:109B90000948E43801680D4A01F4E06111430160AD
:109BA000BFF34F8F00BFFDE72C13002046617461A7
:109BB0006C206572726F7200F0ED00E0537973747F
:109BC000656D207265736574000000000400FA057D
:109BD0000EB500210091CDE901106A4644F2010062
:109BE000FFF7B8FF0EBD0000074B9B7823B12AB1E9
:109BF00020B10068037C1BB1082070470720704724
:109C000041744261002070479414002070B502F046
:109C1000D9FB104800240B21047044700E4D817054
:109C200014206C602C706C70FFF7E8FC0721142086
:109C3000FFF705FD1420FFF7ECFC0848046007213E
:109C40001120FFF7FCFC0548001F0068A8600020F9
:109C500070BD0000941400208012002008150140FF
:109C60002DE9FC47DFF8789099F8023073B368B3B8
:109C7000052902D20720BDE8FC87436933B3437C42
:109C8000012B25D0002704460025884616468DF86E
:109C90000050684600F038F801A802F015FFC8B17E
:109CA000012101700F4944600968C0E90218C0E948
:109CB00004769DF8040089F801009DF8000000F08A
:109CC00047F81420FFF7B0FC2846D4E70820D2E775
:109CD0000F46D8E704259DF8000000F039F8F3E7B7
:109CE00094140020041501400649897839B130B137
:109CF000416921B100210174022102F067BD0820F1
:109D0000704700009414002030B5EFF3108172B654
:109D10000D4A9468012324B10370002900D162B672
:109D200030BD93604FF0E023D3F88051074C2540BD
:109D30001560C3F88041D3F8844154605A17C3F8C2
:109D4000842100220270E8E7A0150020FC06FFBD78
:109D50000B498A68002A11D000280FD1EFF3108038
:109D600072B60B684FF0E022C2F800314B68C2F8BF
:109D7000043100228A60002800D162B670470000DA
:109D8000A01500202DE9F041064608680C46411C4C
:109D90004FF0A0474FF0010506D005FA00F1C7F8D3
:109DA0000815206801F064FA6068411C02D00021A7
:109DB00001F055FA3168A069C1F82405607D217D64
:109DC00032680843C2F86C05D4E900123068C0F864
:109DD0000C15C0F81425207D012815D1A068411C60
:109DE00002D0002101F03BFAE068411C05D085401B
:109DF000C7F80855E06801F03BFAD4E90212306870
:109E0000C0F80825C0F81015BDE8F0812DE9FC4721
:109E1000002517880646158090F82D0014468946BF
:109E200030B13A462146484600F0B1F8051E09D146
:109E3000B0784FF00C0A18B32088C846001DB8420D
:109E400002D95046BDE8FC87684679DF0028F9D181
:109E50002088032108F8001020881921401C80B2B6
:109E6000208008F800102088401C80B2208000EB81
:109E70000801BDF8000002F0C7FD218808442080D9
:109E8000F0780222C8B1218896F9033001F1030C61
:109E90004846BC45D5D8425421884FF0010C491C96
:109EA00089B2218000F801C02188491C89B2218033
:109EB00009F801302088401C20807068B8B12188E2
:109EC00090F9003001F1030C4846BC45B9D8425422
:109ED00021880A22491C89B2218042542188491CC8
:109EE00089B2218009F801302088401C2080308907
:109EF00050B1CDE900474B460622022106F1080089
:109F000002F0FAFD051E9DD1308A50B1CDE900471F
:109F10004B460722032106F1100002F0EDFD051E5D
:109F200090D1308B50B1CDE900474B46152214211A
:109F300006F1180002F0E0FD051E83D1306A30B151
:109F40003B462246494600F087FB051EDBD1706A7E
:109F500030B13B462246494600F07EFE051ED2D176
:109F600096F82C0038B13B4622464946304602F06E
:109F7000E1FA051EC7D1307838B13B462246494642
:109F8000304600F0EFFE051EBDD128465AE77CB5ED
:109F9000054608880C460930904201D90C207CBD4A
:109FA00068466DDF0028FAD121880820685420888F
:109FB0001B21401C80B2208029542088401C80B284
:109FC00020802844DDF801100160BDF80510818073
:109FD0002088801D80B220809DF80010490800D0A4
:109FE000012129542088401C208000207CBD0000D5
:109FF0002DE9FC410646C0074FF000050ED0104F7A
:10A0000000240122385D009500231146019501F0DE
:10A01000E7F8641C042CF4D300F046F8B0070DD523
:10A02000074E0024361D0022305D032300951146A3
:10A03000019501F0D5F8641C042CF4D3BDE8FC8133
:10A04000C6CB010007490B5C4FF0A041D1F80425B5
:10A050000120984020EA0203C1F808351040C1F8F9
:10A060000C057047C6CB01000249085C012101F0D4
:10A070001AB90000C6CB01000249085C002101F0BA
:10A0800012B90000C6CB01000649095C4FF0A040A0
:10A09000D0F80405C84010F0010000D0012080F085
:10A0A00001007047C6CB010010B500242046FFF721
:10A0B000DBFF641C042CF9D310BD10B5002420462E
:10A0C000FFF7DAFF641C042CF9D310BD10B502466B
:10A0D000064B4FF0FF3000215C5C944201D10846F2
:10A0E00010BD491C0429F7D310BD0000CACB0100E4
:10A0F0002DE9F0470D468146FFF7E8FF04460428A6
:10A1000036D2DFF874801B481C4EA8F10C0725B32B
:10A11000012D0ED0022D2BD104EB440030444578A4
:10A12000002D25D0B968002922D02846BDE8F04787
:10A13000084704EB4401755C0E44717849B10E4A3E
:10A140004FF40041093A8068FFF78AFD08B987F8A3
:10A150000390B17808F80410E2E78068FFF7C4FDC7
:10A1600004EB4401314418F804008D78A842D7D09C
:10A17000BDE8F087D0CB010048120020B4130020C6
:10A1800070B50023042810D20D4D00EB4004012AC5
:10A1900002D101290CD00022094E00EB40003044CE
:10A1A00061B1012906D0022906D00723184670BDE7
:10A1B0000E30C2B22A55F9E74270F7E78270F5E730
:10A1C000B4130020044A014600201279D20702D0BD
:10A1D000084600F04DB870473C12002070B50646A6
:10A1E0001E480024C0E90161B00720D500250122E6
:10A1F00011462846FFF7C4FF6D1C0446042D02D209
:10A20000002CF4D013E094B940F2666204211448A3
:10A21000FFF764FC04000AD1FFF74EFC040006D1EE
:10A220000F48104A0021001FFFF7DEFC0446F0072C
:10A2300012D00120FFF7DCFE74B909480A4A002158
:10A240000C38FFF7D1FC040006D10548074A01216C
:10A250000838FFF7C9FC0446204670BD3C120020B8
:10A26000DCCB0100EDA40100F5A90100B19A0100C9
:10A270002DE9F05F6A4C054600266078B34618B1B8
:10A2800084F801B000F09EFB664F4FF47A694FF4FA
:10A29000C87A4FF00108182D62D2DFE805F0AC0C47
:10A2A0000C31404D62676B746B74BE7D7D7D7D7D2E
:10A2B000ACAFB2B5BEBE0020FFF7E6FE00284FF0FF
:10A2C000000008D0FFF7D0FE022D02D14FF4E1606C
:10A2D00008E0484606E0FFF7CFFE022D01D1C82076
:10A2E00000E05046410CC0034FF4FA72801841F16F
:10A2F0000001257052000023FFF710F801462AE004
:10A300000020FFF7C1FE00284FF0000004D0FFF747
:10A31000ABFE4FF44870E5E7FFF7AEFEDFE7002045
:10A32000FFF7B2FE00284FF0000002D0FFF79CFEBE
:10A33000CFE7FFF7A1FED4E70020FFF7A5FE002836
:10A340004FF0000002D0FFF78FFE01E0FFF794FE10
:10A35000257041F69A1100223868FFF781FC064605
:10A3600046E00020FFF76EFE257008E0002051E077
:10A3700025703DE084F801800120FFF763FE002294
:10A3800040F6CD41E8E784F801800120FFF75AFE4E
:10A3900000224FF48041DFE77868FFF7A5FC06460E
:10A3A000D5F1110000D02EB10220FFF75DFE84F838
:10A3B00002B01DE0012816D980B2C8214843C11758
:10A3C000C90341EA5041C0034FF4FA72801841F1C9
:10A3D000000152000023FEF7A1FF01460022786829
:10A3E000FFF73EFC06460220FFF746FE84F8028097
:10A3F0003046BDE8F09F00F0E5FAB9E700F0E2FA78
:10A40000B4E700F0DFFA04E000F0DCFA0020FFF728
:10A4100033FE0120FFF730FEAAE7FFF74EFEA7E765
:10A420003C120020D0CB01002DE9F8430546861CE4
:10A4300000208DF8000090460F464FF00109684655
:10A44000FFF762FC1B4C20683860D4E90001401A19
:10A45000A16804F21C47081A0EE00121384600F0FA
:10A46000D5FC00F04DFB0146384600F0CFFCD4E9A6
:10A470000001401AA168081A401C8642EDD8B8F1C4
:10A48000000F03D0052065F3891002E0062065F374
:10A490009F50A2682168114004EB8101C8602068C8
:10A4A000304420609DF80000FFF752FC4846BDE8AC
:10A4B000F8830000B816002030B482680468531C8A
:10A4C0008360A154D0E901128A4202D330BC00F06B
:10A4D0008EBD30BC70470000034803C8814201D1E3
:10A4E0000120704700207047B81600200078022134
:10A4F000FFF7FEBD05494FF0FF32082841F8202044
:10A5000002D3084480F8482070470000F41300206C
:10A51000F0B54FF0FF3512B10023082601E0082303
:10A520000C260C4C05E000BF54F823707F1C04D0AF
:10A530005B1CB342F8D32846F0BD26185DB286F8FE
:10A54000305044F82310002AF5D1E11881F8480072
:10A55000F1E70000F41300200249084490F93000AC
:10A5600070470000F413002070B5084C050009D0B6
:10A5700010342168002907D00868206049682846FF
:10A580008847F6E70834F4E770BD0000E0130020C8
:10A59000054A012120B1012805D19170FFF7E4BFE0
:10A5A00051700020FAE77047E01300202DE9F05FBA
:10A5B00026484168F1B3DFF898B00E688146DBF8B1
:10A5C000004087688078E11B21F07F45ED1CB0B921
:10A5D000DFF880804FF48030C8F84403C8F80403E3
:10A5E0001120FFF70BF81120FFF713F84FF0010AC5
:10A5F000C8F800A02F2001F065FC89F802A0B54240
:10A6000000D23546124BE8193C3320F07F401860E9
:10A61000DBF800105A46091B21F07F41001B20F097
:10A620007F40C91C81420FD9106818602F2001F0AB
:10A6300049FC00E004E0BDE8F05F1120FEF7F4BF44
:10A64000BDE8F05F01F0BEBEBDE8F09F80120020C3
:10A6500004150140001001402DE9F041178806461D
:10A66000B81D14460D46984202D90C20BDE8F08171
:10A670003188072206290AD34FF4486C4FF6FF733E
:10A68000614501D9994202D17088062801D210464D
:10A69000ECE7604501D99842F9D1994203D098423C
:10A6A00001D08142F3D80520E85520881221401CB2
:10A6B00080B2208029542088401C80B2208041191B
:10A6C000308802F0A1F92188084480B22080411925
:10A6D000708802F099F92188084420800020C5E79D
:10A6E0002DE9F0470025DFF88C803CE06068002110
:10A6F00000EBC506012032789146FEF740FED4E912
:10A70000062300EA020701EA030C57EA0C0728D0E7
:10A7100082438B434846C4E9062301F095FC327816
:10A720008246914601200021FEF729FED4E9042348
:10A7300000EA020401EA03074A4650460021FEF7F8
:10A740001EFE44404F403C430BD17078012801D09D
:10A75000012100E00021726881EA0A010AB148463D
:10A7600090476D1CEDB298F8000044468542BDD379
:10A77000BDE8F0876012002010B50021024800F00B
:10A7800050FB80F3100010BDD41A00200E4910B504
:10A790000A784C780023A24212D0521CD2B20A701E
:10A7A000022A00D10B70084A0B780C3252F8232091
:10A7B00002608868104420F07F408860012010BD4E
:10A7C0000360002010BD0000801200202DE9F04140
:10A7D0008046024601200021FEF7D1FD1A4F0546B2
:10A7E0000E467868FFF780FA00280CD1174CD4E9A0
:10A7F000062110462A4001EA06031A4305D0A84361
:10A80000B143C4E90601BDE8F081404601F01CFCFB
:10A8100030B1D4E9040128433143C4E9040105E01F
:10A82000D4E90410A943B043C4E90410D4E90601F3
:10A8300028433143C4E90601A1687868BDE8F041C6
:10A840000022FFF70DBA000004CC010060120020C6
:10A850002DE9FC5F0E008346DDE90C47C6F10000E0
:10A8600098469246814600D40846012503E000BF81
:10A8700090FBFAF06D1C5045FADAA84500D9454620
:10A8800024B1002E01DB780700D5641EB80702D57D
:10A89000B8F1000F0AD0F80708D13CB1A54205D2A3
:10A8A00020215846641EFFF707FEF6E7002E02DA65
:10A8B0004E462D2102E0780703D52B215846FFF79D
:10A8C000FBFD07F0030002280BD1B8F1000F08D1FF
:10A8D0003CB1A54205D230215846641EFFF7ECFD7D
:10A8E000F6E7CDE90047434652463146584602F066
:10A8F00091F8BDE8FC9F000070B50D460446006865
:10A900004FF4887101F0A3FA4FF49071206801F0C0
:10A910009EFA4FF49271206801F099FA4FF4A271F7
:10A92000206801F094FA20681249C0F804132068E6
:10A930006907000B40B2090E002806DA00F00F008C
:10A9400000F1E02080F8141D03E000F1E02080F821
:10A95000001420680121000B40B200F01F0291405A
:10A960004009800000F1E020C0F88012C0F800111A
:10A9700070BD000010030200024600201268930719
:10A9800002D0530702D47047500714D502F00300D9
:10A99000012802D002280CD105E0C2F383100B6815
:10A9A000801C184404E00223086803EB9252104410
:10A9B000086001207047086800EB9253C2F38910C9
:10A9C000401CEEE70A4810B5807860B1002401E031
:10A9D000022C06D02046FFF747FB641C042CF7D35B
:10A9E00010BD0324F6E7BDE81040FFF75DBB000093
:10A9F0003C12002003480179C90702D00078FFF714
:10AA000037BC70473C1200202DE9F047394E002733
:10AA100080463D46DFF8E090D6F804A057E003D02A
:10AA20000446D0F81C8035E099F8002002EB420182
:10AA3000521CD2B289F8002009EBC10199F802300A
:10AA4000091D9A4201D189F8005048680A780446E5
:10AA5000012A12D0022A02D0032A3BD108E001F0D9
:10AA600085FE00B10127257434E00574C06900E05B
:10AA700070680028F9D170602CE0207C50BB886899
:10AA80006060C868A0600869E0604869A061F0780B
:10AA900000B165606268B168184B501A20F07F40C1
:10AAA000984202D2A168084406E0881AA16820F002
:10AAB0007F40814202D9081A206000E0256065606D
:10AAC0000120A56020742046E56101F031FEB8F157
:10AAD0000000A4D199F8001099F801008142A3D197
:10AAE00017B97168514502D00120BDE8F0870020F8
:10AAF000FBE700008012002094140020FFFF7F007D
:10AB00002DE9FF410026234800F07DF92148001F70
:10AB1000074600F078F9204C60680090A56800E0D6
:10AB200000986946284004EB80000C30FFF724FFB2
:10AB30000028F5D101AA009901EA050304EB83037B
:10AB4000491CDB6842F82030401C00910228F2D3F7
:10AB5000019800F0030001280BD0022810D10198C1
:10AB6000032101EB90500099BDF80A6001EB9000C1
:10AB700005E00198BDF80A60C0F383100844009016
:10AB8000384600F03DF908B10098606004B03046E6
:10AB9000BDE8F081D01A0020B816002008B54FF4A7
:10ABA0000041002000F0F8FD08B1FFF711F800F0B7
:10ABB0006BFCFFF72BF808B1FFF70AF80021012022
:10ABC000FFF70CFB08B1FFF703F800F003FF08B133
:10ABD000FEF7FEFF01F06AF808B1FEF7F9FF00206A
:10ABE00000906946012000F01DFF08B1FEF7F0FF5C
:10ABF000684600F097FF08B1FEF7EAFFFEF71EFF78
:10AC00000D480321008801EB00400CA100F05AFD23
:10AC100010480121007873DF08B1FEF7D9FF022048
:10AC2000FFF7D0FA08B1FEF7D3FF00F03BFC002895
:10AC3000FBD100F0E3FEF8E72C13002042656163CE
:10AC40006F6E206578616D706C65207374617274CD
:10AC500065642E001012002070B5144682880E46DE
:10AC600005462088111D0144921C994201D8FE2AF4
:10AC700001D90C2070BD521C32542088FF21401C89
:10AC800080B2208031542088401C80B220808119FD
:10AC9000288801F0B9FE2188084480B22080AA8863
:10ACA00042B1A96841B13044FEF77CFB2088A988F5
:10ACB00008442080002070BD072070BD2DE9F047BA
:10ACC000C7880446181D16468946B0FBF7F1B0FB4D
:10ACD000F7F207FB12009A193A44D21CB2FBF7F2C2
:10ACE000DDF820A001E02468491E0029FBD13D1AAF
:10ACF0008846B54216D818E0BAF1000F05D02118E1
:10AD000009EB08002A46091D04E0204409EB08016C
:10AD10002A46001DFEF746FB00202468761BA84447
:10AD2000B74201D9354600E03D46002EE4D1BDE8EA
:10AD3000F087000030B5024659B100F059FD0021FE
:10AD4000074C09E004EB810315685B88AB4202D134
:10AD50001160002030BD491C8142F3D3052030BD75
:10AD600010130020F8B50F46017814460546012956
:10AD700001D1687830B12088821C9A422DD80129EF
:10AD800002D006E00720F8BD69780144891C994289
:10AD900023D8181A801E86B2ADF800602188B81C2E
:10ADA000084469467DDF0028EDD12878022805D1C6
:10ADB000BDF80010B14201D809210AE0082101289C
:10ADC00005D16878B04202D8ADF8000001E0ADF8D6
:10ADD0000060BDF80000FE2801D90C20F8BD2288D3
:10ADE000401CB8542088401C80B2208039542088F0
:10ADF000401C2080BDF80010084420800020F8BDD1
:10AE0000002100F009B8012100F010B808B56A4629
:10AE1000FEF733FA009808BD08B56A46FEF713FA44
:10AE200008BD08B56A46FEF7F5F908BD08B56A46DB
:10AE3000FEF7FCF9009808BD08B56A46FEF72AFA45
:10AE4000009808BD38B5044600258DF800506846C6
:10AE5000FEF75AFF21686268086890420ED9401ECA
:10AE600008600178A38AE26801FB0325227A216841
:10AE7000101AC0B20A79824200D208719DF800000F
:10AE8000FEF766FF284638BD38B5054600208DF828
:10AE900000000C466846FEF737FFE868A98A201ACA
:10AEA000B0FBF1F12A681068431C136001709DF833
:10AEB0000000FEF74DFF38BD10B530B1017A426891
:10AEC0000368891AC9B21A6006E00E2010BD036833
:10AED0001A68541C1C601170491EC9B2F7D2006870
:10AEE00000210171084610BDC20800F007030120CF
:10AEF000895C98400840704710B5C20800F007030D
:10AF0000885C01249C402043885410BD00F180409F
:10AF10000068002800D00120704708B500F180408B
:10AF2000002101600068009008BD000070B50B4C66
:10AF3000207808B185250FE00020A06060602061C6
:10AF4000E060074800F0A0FF054600F009FF08B9DF
:10AF500000F084FF01202070284670BDE01300201F
:10AF600091A5010038B500258DF800506846FEF720
:10AF7000CBFE074CE068401EE060E06810B900F0CE
:10AF800093FFA5709DF80000FEF7E2FE38BD0000BB
:10AF9000E013002070B5064604780C4888B01546CA
:10AFA00040F82420094A0869121D42F82400202292
:10AFB0006846FEF7F7F904940DB1054A00E0002257
:10AFC0006946301D01F098F808B070BD4C120020A1
:10AFD000E5C801000FB408B50399002904D004AAFC
:10AFE00000926A4600F00FF801B05DF814FB10B54E
:10AFF00082680446002A05D0D4E9040321689847F2
:10B000000020A06010BD2DE9FC4791460C00804651
:10B0100076D014F8011B39B125290ED04046FFF730
:10B020004BFA20780028F4D198F80C00002867D05B
:10B030004046BDE8FC47FFF7DABF00200122217837
:10B040002B291BD02D2902D0302908D102E040F055
:10B05000010001E040F00200641C002AEFD100254D
:10B060002A290ED02178A1F130020A2A11D205EB4B
:10B07000850201EB4205641C303DF1E740F004001D
:10B08000EAE7D9F800100B1DC9F800300968641C04
:10B090000D44217800232E290BD114F8011FA1F1B2
:10B0A00030020A2A05D203EB830201EB4203303B54
:10B0B000F3E76C290DD068290BD0692921D00BDC6E
:10B0C000252918D0582931D063290ED0642915D1EB
:10B0D00017E014F8011FECE7702969D0732932D00A
:10B0E00075291BD0782909D120E0D9F80000011D6D
:10B0F000C9F8001001784046FFF7DEF9641C90E7BC
:10B100006CE0D9F800100A1DC9F800200968CDE9E3
:10B1100000500A224046FFF79BFBEFE7D9F80010EA
:10B120000A1DC9F8002009680A2206E0D9F80010B3
:10B130000A1DC9F8002009681022CDE900504046D8
:10B1400001F068FCDAE7D9F8001000270A1DC9F8F9
:10B1500000200E68C00705D112E04046761C7F1C17
:10B16000FFF7AAF931780029F7D104E02021404601
:10B170006D1EFFF7A1F9BD42C0D9002DF6D1BDE784
:10B180004EB13046FEF732F9074604E02021404632
:10B190006D1EFFF791F9BD4206D9002DF6D103E0EF
:10B1A0004046761CFFF788F931780029F8D1A5E7E9
:10B1B000D9F80000011DC9F800100568302140468B
:10B1C000FFF77AF978214046FFF776F90820002149
:10B1D000CDE90001034610222946B0E7BDE8FC870F
:10B1E00070B541EA4201DDE904564FF0A04441EA5E
:10B1F000830141EA052104EB800041EA0641C0F8E1
:10B20000001770BD70B541EA4201DDE904564FF008
:10B21000A04441EA830141EA052104EB800041EAB0
:10B220000641C0F8001770BD70B541EA4201DDE982
:10B2300004564FF0A04441EA830141EA052104EBA2
:10B24000800041EA0641C0F8001770BD1CB500211E
:10B2500000910B4601220191FFF7E6FF1CBD1CB5D2
:10B2600000220B46009211460192FFF7DDFF1CBD44
:10B270001CB5002100910B46012201911146FFF7F8
:10B28000D3FF1CBD4FF0A04202EB8000D0F8002796
:10B2900022F44032C0F80027D0F8002742EA0141EA
:10B2A000C0F80017704701224FF0A043824011B14F
:10B2B000C3F808257047C3F80C25704718B5084B2C
:10B2C0006C4601441B68009306E000BF54F8203030
:10B2D000D3F81035401C08C28142F7D818BD0000D1
:10B2E000FCCB0100034908B5084400210160006857
:10B2F000009008BD0060004002494058012800D07D
:10B30000002070470060004030B5124B014600201D
:10B31000D3F81044224609E0157A854205D1401C35
:10B320000A28F7DB4FF0FF3030BD5268002AF3D116
:10B33000421CF9D00872D3F810242AB152684A602E
:10B34000D3F81024516030BD0022C3F810144A60B5
:10B3500030BD0000B8160020F0B595B01C4615466B
:10B360000F4608461A9E00F013FB182109A8FEF7A5
:10B3700032F80E96CDE909540023082203A9384675
:10B3800000F01BFB05980690BDF81000ADF81C00FE
:10B39000BDF81200ADF81E0000208DF821000398C2
:10B3A000082600F00300012802D0022818D032E05D
:10B3B00003983346850AC0F3C2008DF82000039835
:10B3C0000FA9C0F38314A200384600F0F6FA09A8CA
:10B3D000009006AB22460FA9284600F035FA1AE085
:10B3E0000398840DC0F3C2008DF82000082C01D210
:10B3F000254600E0082533462A460FA9384600F0C6
:10B40000DCFA2E44641B09AB06AA29460FA800F0FB
:10B410006DF9002CEAD1384600F0C0FA15B0F0BD45
:10B420007047012001F036BA10B5044800F0F0FE74
:10B43000BDE81040002001F02DBA0000A412002049
:10B4400008B5034A00924023024AFFF785FF08BD72
:10B4500009C50100B81500200A4A012902EBC00005
:10B4600007D0022907D0032907D0042907D00020DC
:10B470007047022070470420704700797047407978
:10B480007047000040D5010010B5FFF7CAFF042146
:10B490000348FFF739FF02490120487210BD000040
:10B4A000AC1200202DE9F04F8DB0FFF715F818B160
:10B4B00000200DB0BDE8F08F7A4C4FF0000BC4F8BF
:10B4C00018B4BFF34F8F60680290A568D846284033
:10B4D00004EB800008E021680298814201D8616095
:10B4E000E6E7284004EB80000C3002A9FFF744FA9D
:10B4F0000028F0D105AA029901EA050304EB8303B1
:10B50000491CDB6842F82030401C02910228F2D32B
:10B51000059800F00300022802D001284ED0A9E0CF
:10B5200005985022810D8946B2EB905F00D85021DA
:10B530000E4666F39F50059008315B4800F0DFF936
:10B54000070079D000F024FA4346082205A93846BE
:10B5500000F039FA029908F1080A2940681A8000B7
:10B56000001D864223D94F4D0C3530B1C2B204EBD9
:10B570008101301A90460C3104E02946F2B20025D0
:10B5800090462846C6B25346384600F01CFA0AEBED
:10B5900008032DB1324629464FEA070000F013FA9E
:10B5A000029909F1030001EB900002903BE004EBEB
:10B5B00081015346324638460C31EFE70598C0F317
:10B5C0008310062800D30620059960F38911C1F382
:10B5D0008310801C05918100334800F090F907002A
:10B5E00048D000F0D5F94346082205A9384600F0B6
:10B5F000EAF908F1080800260FE00298434600EA3D
:10B600000501401C04EB81010290042238460C31F4
:10B6100000F0D9F908F10408761C0598C0F38310EE
:10B62000B042EAD847B1D4F81054D4F8180468B13D
:10B63000384600F0B3F92FE01CE0687A012804D105
:10B640002A6828463946126890476D68002DF4D163
:10B65000384600F0A3F98DF800B06846FEF754FBB9
:10B66000D4F8180408B9029860609DF80000FEF74D
:10B670006FFB11E0D4F8104404E02168204689688B
:10B6800088476468002CF8D108480221008801EB43
:10B69000004007A100F016F8FEF71EFF80F0010041
:10B6A00007E70000B816002098D501002C130020F1
:10B6B0004261636B656E647320666C757368656464
:10B6C0000000000000231A4600F0ACBF08B50123BB
:10B6D00000926A4600F0A6FF08BD1CB5CDE9002324
:10B6E00002236A4600F09EFF1CBD00002DE9F047D2
:10B6F0000E4680461C46924608293ED894F80C9087
:10B70000002020731946104600F010FE0025B542B7
:10B7100006D218F805201AA12046FFF75BFC03E0CB
:10B7200019A12046FFF756FC6D1C082DEFD317A179
:10B730002046FFF74FFC0025B54210D218F80570DF
:10B74000FDF72CFE0068C05D10F03E0F01D03A46B8
:10B7500000E02E220EA12046FFF73CFC03E00DA1E5
:10B760002046FFF737FC6D1C082DE5D3012221464A
:10B77000504600F0BDFD84F80C90BDE8F087000055
:10B780002025303278000000202020007C000000BE
:10B790002563000020000000104810B5FF218160E3
:10B7A000002101604160C0F81814C0F8141480F83A
:10B7B00020140B4800F0F0F800280DD109480A4980
:10B7C0000A4B401AC108002003E000BF23F8200004
:10B7D000401C8842FAD3002010BD0000B81600209B
:10B7E00098D5010098D5010040D501001013002024
:10B7F00002480349401AC0087047000098D501006C
:10B8000040D5010013B56846FFF794FA08B100204F
:10B810001CBD0248009950F831001CBD40D5010004
:10B8200070B508480125D0F8104480F8205405E090
:10B83000657221682046496888476468002CF7D102
:10B8400070BD0000B81600202DE9FF4781460C9D11
:10B8500000200C462F7B287398461646294618462A
:10B8600000F064FD072E42D2DFE806F004090F164F
:10B870001F2A360049462846FFF7ACFB37E0494609
:10B8800028462268FFF7A6FB31E0D4E900234946A9
:10B890002846FFF79FFB2AE0A0680090D4E9002328
:10B8A00049462846FFF796FB21E0D4E90201CDE99D
:10B8B0000001D4E9002349462846FFF78BFB16E038
:10B8C00004F1080007C88DE80700D4E900234946C1
:10B8D0002846FFF77FFB0AE004F108000FC88DE857
:10B8E0000F00D4E9002349462846FFF773FB0022E6
:10B8F0002946404600F0FCFC2F73BDE8FF872DE988
:10B90000F041858A80462D1F4819C01CB0FBF5F018
:10B91000C6B24046FFF796FA041E19D000202071E7
:10B9200001206071E58000272546761EC4F800805E
:10B930000BE04046FFF786FA60B16179491C6171FE
:10B94000286005467F1CC0F80080B742F1D320462E
:10B95000BDE8F081204600F002F80020F8E72DE96C
:10B96000F041457901466B1E002201E00968521C36
:10B970009A42FBD30F680146002605E038460C6862
:10B98000FFF782FA2146761CAE42F7D3BDE8F0817C
:10B990000121001DFFF73ABAFFF78EBA10B5044631
:10B9A0000121001DFFF748FA10F0FF0F04D12046D7
:10B9B000BDE81040FFF7D3BF10BD38B50124009497
:10B9C000FFF77CF938BD38B500240094FFF776F90D
:10B9D00038BD0000064910B500204870091D0860F8
:10B9E000BFF35F8F0349044800F0DEF9002010BD6B
:10B9F000941200203CCC0100AC15002010B500F0E2
:10BA0000AFF908B141DF10BD20BF40BF20BF10BD5E
:10BA100020B1034909680160002070470E2070477B
:10BA200028CE0100FEB502460D460846FFF7F0FF9E
:10BA3000002869D1002400940194012606208DF885
:10BA40000020ADF8040002948DF8026069462020C1
:10BA50002A6869DF2D4F48B100F0EAF939880246BB
:10BA600006EB01432A491846FFF730FE0094019483
:10BA700002948DF80140694640202A6869DF48B188
:10BA800000F0D6F93988024606EB014321491846F1
:10BA9000FFF71CFE0094019402948DF80040694663
:10BAA00001202A6869DF40B100F0C2F902463888F7
:10BAB000194906EB0040FFF709FEF82000900194B9
:10BAC00002946946A1202A6869DF48B100F0B0F904
:10BAD0003988024606EB014310491846FFF7F6FD88
:10BAE0000094019402948DF800406946A0202A68D1
:10BAF00069DF40B100F09CF902463888084906EB3E
:10BB00000040FFF7E3FD0020FEBD000034130020DD
:10BB100024D401006CD4010084D30100D0D30100EF
:10BB200030D301002DE9F0410446D0F8008060DFF9
:10BB30002168194D074641451CD92888022606EB85
:10BB4000004016A1FFF7BEFD2888424606EB0040E4
:10BB50001EA12368FFF7C1FDF006D0F80C01216893
:10BB6000800200F10050421A288825A106EB00400F
:10BB7000FFF7ACFD012467B1384600F059F90246E1
:10BB800028882AA104EB0040FFF7A0FD3846BDE855
:10BB9000F0812E480470F9E734130020496E737564
:10BBA0006666696369656E742052414D20616C6CF4
:10BBB0006F636174656420666F72207468652053DA
:10BBC0006F66744465766963652E00004368616E34
:10BBD0006765207468652052414D207374617274EA
:10BBE000206C6F636174696F6E2066726F6D2030B8
:10BBF00078257820746F20307825782E000000009A
:10BC00004D6178696D756D2052414D2073697A657B
:10BC100020666F72206170706C69636174696F6E09
:10BC200020697320307825782E00000073645F62ED
:10BC30006C655F656E61626C65282920726574753C
:10BC4000726E65642025732E000000000B13002027
:10BC500030B5144891B00078002820D05FF034054A
:10BC6000ADF8405010A903A861DF30B1052816D007
:10BC700011B0BDE83040FDF7ABBF03AC0A496846E0
:10BC800000F092F807E000BFD0E90021204690477D
:10BC9000684600F0A0F802980028E1D0F4E711B05F
:10BCA00030BD00000B1300202CCE01007CB5204CD1
:10BCB000207808B108207CBD0120A070002000F091
:10BCC000F5FB112819D0002000F008FC19480026C7
:10BCD000006801908DF800606846FEF715F8164977
:10BCE00001A810DF05000AD0002020709DF8000098
:10BCF000FEF72EF82DB128467CBD00207CBD01202A
:10BD0000F3E7A67066700721162000F085FB08B1E6
:10BD1000FDF75EFF0721152000F07EFB08B1FDF75F
:10BD200057FF00F057FC012000F0D8FBE5E70000CA
:10BD300008130020C0CD0100559B01000EB5074936
:10BD4000684600F031F805E0D0E900108847684601
:10BD500000F041F802980028F6D10EBDDCCD0100BC
:10BD60000148007870470000081300201FB568469E
:10BD70004BDF30B1052814D004B0BDE81040FDF70A
:10BD800027BF084901A800F00FF806E0D0E900211C
:10BD90000098904701A800F01EF803980028E6D00C
:10BDA000F4E71FBD48CE0100016009684160AFF3B0
:10BDB000008010B5D0E900215368994201D10021DB
:10BDC00004E0D1E90034A34202D01946816010BDDD
:10BDD00008314160F0E7816800290BD00268926861
:10BDE0000A44826041684B689A4203D1083141603D
:10BDF000FFF7DFBF704700000C4A10B502F59473DF
:10BE00000EE0991AC91001EBD171491002EBC10182
:10BE10000C68844201D90B4602E005D201F1080208
:10BE20009A42EED3002010BD486810BD5CCC0100E2
:10BE300000B5FFF7E1FF002800D1014800BD000078
:10BE400048CC01004058002800D00120704708B5B8
:10BE5000002242504058009008BD00000848006889
:10BE6000012110F0010F08D14FF0E020E02280F80E
:10BE70000024C0F88012C0F8001102480160704729
:10BE800000E100E0180500400649024600200B7959
:10BE90000BB1852070470A6001220A7100224A71A5
:10BEA0007047000054120020044901200860044833
:10BEB0000168C1F300410029FAD170470C0000402D
:10BEC00018040040002802D001498001084770474B
:10BED0000DCC01002DE9F0418846054600F0F0F94F
:10BEE000234E002828461AD0FEF736FB304490F83F
:10BEF00048008009032802D001280ED007E04FF047
:10BF0000A040D0F81005E84010F0010F05D0032143
:10BF10002846BDE8F041FFF7B5B90221F8E700F087
:10BF2000DBF9002822D02846FEF716FB04464FF422
:10BF3000807000EB84000F4F81B207EB8400D0F8D3
:10BF4000102542F00102C0F810250846FFF7CAF993
:10BF5000B8F1000F0AD02846FEF7FEFA56F8200086
:10BF6000002803D00120A040C7F80403BDE8F081F9
:10BF7000F4130020006000402DE9FC41DFF8BC8094
:10BF8000044608EB0400002790F930001346C01760
:10BF90000E46401C01D008274CE0B0781946C0F38B
:10BFA00040022046FEF7B4FA0546401C41D0B07866
:10BFB000410719D4C0070AD04FF0A04000EB84011C
:10BFC000D1F8000720F00200C1F8000707E00021C7
:10BFD0007378204600910A460191FFF713F917493B
:10BFE00020465431FEF788FFB078800718D51448F2
:10BFF000317800EB8500D0F81025124B1A40C0F8BC
:10C0000010254FF4F8524FF4403302EA042203EAB9
:10C0100001410A43D0F810150A43C0F8102509E081
:10C0200008EB0500327810F8481F41EA82110170D0
:10C0300000E004273846BDE8FC810000F41300202E
:10C0400000600040FFE0FCFF4FF0A041D1F8101568
:10C05000C14011F0010000D00120704770B5184DAB
:10C0600095F8580008B1082070BD0020411E2A181C
:10C07000401CC0B282F830102028F8D3002420469B
:10C08000FEF738FA641CE4B20C2CF8D300240D49F6
:10C09000E0206C6581F8000401264020891FC1F86A
:10C0A0008002C1F800014FF4BE70FFF71BF906498A
:10C0B000F007C1F8040385F85860204670BD000001
:10C0C000F413002006E000E000600040034890F810
:10C0D0005800002800D0012070470000F413002011
:10C0E0000121B1EB507F01D1012070470020704742
:10C0F00000207047704700002DE9F04105461646C4
:10C1000000790F46154A00EBC00102EB810494F858
:10C11000201011B10820BDE8F081114951F820101C
:10C120002868FFF7E5FF08B11120F4E739462846F3
:10C13000FDF728FE6660386920601EB1397F284609
:10C14000FEF7DAFB28680821C0F800150020A0617E
:10C15000E0610121606184F82010DCE750140020C8
:10C1600000CC01002DE9F04704460E460079204935
:10C1700000EBC00001EB800517463046FFF7B0FF2B
:10C1800030B1204600F036F820B11120BDE8F0872C
:10C190001020FBE76F61AE604FF4907600273146C8
:10C1A0002068FFF754FE4FF4AC7841462068FFF753
:10C1B0004EFE2068AA686969C0F84425C0F8481591
:10C1C000206801218160686878B9B14649462068D5
:10C1D000FFF738FE064641462068FFF733FE064368
:10C1E000F4D000B10F27002068613846CEE7000088
:10C1F000501400200079054900EBC00001EB8000DD
:10C200004069002800D00120704700005014002031
:10C210002DE9F04704460079274900EBC00001EB07
:10C22000800720684FF00009C0F80095786880B159
:10C2300020682249C0F8081320680121000B40B291
:10C2400000F01F0291404009800000F1E020C0F89A
:10C2500080112068D0F80C25D0F81485D0F8086536
:10C26000D0F810554FF0FF31C0F80C15C0F8141578
:10C270002068C0F80815C0F81015501C02D01046F0
:10C28000FEF7E4FFB8F1FF3F02D04046FEF7DEFFC5
:10C29000681C02D02846FEF7D9FF701C02D0304639
:10C2A000FEF7D4FF2068FFF725FF87F82090C7F836
:10C2B0000490BDE8F0870000501400201003020035
:10C2C0000449084490F93000082801DB0120704738
:10C2D00000207047F41300200449084490F930000E
:10C2E000082801D20120704700207047F413002075
:10C2F00010B50C46017A052908D0407A38B10848B3
:10C3000008A102682046FEF765FE00E01AB106A10A
:10C310002046FEF75FFE2046BDE81040FEF767BEF0
:10C32000E4120020257300000D0A000038B5C38810
:10C330000D46044633B114A0009015A216A128465C
:10C34000FEF748FE217A05291CD0607A48B1A08802
:10C35000FFF782F8164951F8202016A12846FEF76B
:10C3600039FEA0880021FFF74DFA03461049207AD4
:10C37000143951F8202001B02846BDE830400EA104
:10C38000FEF728BE38BD00001B5B306D00000000CA
:10C390001B5B313B33316D0025734C6F6773206439
:10C3A000726F70706564202825642925730D0A005A
:10C3B000E4120020257300003C25733E2025733ACB
:10C3C0002000000070B5012670044FF0E021002528
:10C3D000C1F88001084C4010C4F84803C4F80803B1
:10C3E00066602F20FFF76EFDA660044C2F20A5602D
:10C3F000FFF768FDA57070BD00100140801200209D
:10C400001FB501238DF800308DF808100192D0E996
:10C410000012684690471FBD70B50D460446FDF7F3
:10C42000EFFA70B12846FDF7FDFA68B16807000E13
:10C43000002C0CDA04F00F0101F1E02181F8140D59
:10C4400009E042F2010070BD42F2020070BD04F149
:10C45000E02484F80004002070BD000038B50021FD
:10C46000012548B101280CD0032809D1FFF7F6FCBB
:10C47000BDE83840FEF776BD4FF0E020C0F88051AF
:10C4800038BD8DF800106846FDF73EFC064C20785C
:10C4900008B9FEF74BFDE068401CE060A5709DF810
:10C4A0000000FDF755FC38BDE01300203EB5044602
:10C4B00009496846FFF778FC08E000BFD0E9002191
:10C4C0002046904730B16846FFF785FC0298002867
:10C4D000F4D13EBD11203EBDC4CD01003EB50446A1
:10C4E00008496846FFF760FC07E000BFD0E900217B
:10C4F000204690476846FFF76EFC02980028F5D169
:10C500003EBD0000D0CD010010B5094C0020D2B2D4
:10C51000207004F10800FFF725FE08B1FDF758FB75
:10C520006078002802D021780029FAD010BD0000E0
:10C530009C1200202DE9F0410746806A1446884687
:10C54000C8B3002531E000BFB96A05EB450001EB37
:10C550008006B088801CFE2802D90C20BDE8F0813E
:10C560002288401C08F8020020881622401C80B255
:10C57000208008F800202088401C80B2208000EB3A
:10C580000801308800F040FA2188084480B22080F9
:10C59000B28842B1B16871B14044FCF703FF208812
:10C5A000B188084420806D1CEDB297F82C00A84299
:10C5B000CAD80020D2E7FFE70720CFE7002805D13F
:10C5C0000349012048700020FDF7CEBF70470000EE
:10C5D000E013002010B51620FDF712FA80B10F48C5
:10C5E00090F800044009FDF71DFA60B10C4882681C
:10C5F0004FF480016AB1016841F48001016010BD0F
:10C6000042F2010001E042F20200BDE81040FDF7F5
:10C61000DFBA4FF0E020C0F8001110BD16E000E0D6
:10C62000A01500202DE9F84F204D92468946064678
:10C630009846012269461846AF68FDF7F5FE58B3E3
:10C64000009800210446801C09E000BF00EA0703AF
:10C650005AF8212005EB8303401C491CDA60414550
:10C66000F4D34FEA164AFEF787F84AEA0041601C05
:10C67000384005EB80003C4005EB8402C160D06887
:10C6800066F3C50068F3891069F39F2020F003006A
:10C69000401C20F00400D06095F8200402E000BFA8
:10C6A000FEF700FF0028FBD1BDE8F88FB816002088
:10C6B0002DE9F84F1D4C00256846D4E901A6FEF788
:10C6C00065F8002738B30023009A61681CE0D1F8B0
:10C6D00000C00846944503D9ACEB02020A6015E09D
:10C6E000A2EB0C0263440760D0F80CC0C16981461C
:10C6F000BCF1000F08D006EB030828F07F48C0E922
:10C70000018CC9F81C5005460029E0D1284661601B
:10C71000FEF77AF903E02846FEF776F910B15046A5
:10C72000FDF744FFE770BDE8F88F0000801200209D
:10C730000D4B10B5596831B102680C68A24204D89B
:10C74000A21A0A60C161586010BD0B4603E00B4697
:10C75000C969121B21B10C689442F8D3A41A0C6069
:10C760000260C161D86110BD801200202DE9F04146
:10C77000144E77683D462C4603E0844204D025469B
:10C78000E469002CF9D11BE0D4B1A5420BD1F869C2
:10C79000706040B90C49012088600021B160F070E0
:10C7A0002F20FFF78FFB2168E069E86110B1026874
:10C7B000114401607068874202D00120BDE8F08119
:10C7C0000020FBE780120020001001407CB50646E7
:10C7D00000240D468DF800406846FDF795FA01A843
:10C7E00000F072F970B10570094946609DF80400C7
:10C7F00048709DF80000FDF7ABFA1420FCF714FF19
:10C8000020467CBD04249DF80000FDF7A1FAF7E75F
:10C81000941400202DE9F041194D6C68002C2CD0A7
:10C82000184800270068A968B846401A20F07F46DB
:10C830002068B0420CD82146361A0744E469087CC7
:10C8400020B181F81080886949698847002CEFD1B0
:10C8500029786878814206D1401CC0B268700228ED
:10C8600001D185F80180064869780C3040F82170C4
:10C87000BDE8F0411420FCF7D7BEBDE8F081000010
:10C880008012002004150140014901200870704702
:10C890009C12002010B588B0044620220E4968463C
:10C8A000FCF780FD06200090C01F019002900390CD
:10C8B0004FF0EB7006900CB1084A00E00022694688
:10C8C0000748FEF767FB08B1FDF782F90448001F2F
:10C8D000447008B010BD000090CD010089C801006F
:10C8E000A01200201FB50A4601788DF8001041689B
:10C8F0000191017A8DF80810C0680390044850F83F
:10C900002210001F50F82220684690471FBD0000EB
:10C91000501200202DE9FF410C464FF49277054656
:10C920003946FFF78FFA0026C0B139462846FFF78F
:10C930008EFA02208DF80000D5F88004C5F8800436
:10C940000390D5F83C058DF80800E0680190A661D9
:10C95000E661D4E900126846904723E04FF48877F7
:10C9600039462846FFF76EFAE0B139462846FFF708
:10C970006EFAD5F83C15A069884213D1E06960B120
:10C98000E268D5F8000220F02000C5F80002E06956
:10C99000A0612069E661E06001E0A661E2682046EE
:10C9A000FFF72EFD4FF4A27739462846FFF74AFAE3
:10C9B00060B139462846FFF74AFAA06930B1A6614E
:10C9C000D5F83C152046E268FFF71AFD4FF4907742
:10C9D00039462846FFF736FA002813D0394628464C
:10C9E000FFF735FA606900280CD0D5F84C058DF8B2
:10C9F00000608DF80800A06801906661D4E900121B
:10CA000068469047BDE8FF810870000A4870022020
:10CA1000704700002DE9F05F8346DDE90A4A994638
:10CA200090460D460846012703E000BFB0FBF8F032
:10CA30007F1C4045FAD2B94500D94F465FEACA701B
:10CA400012D18CB15FEA8A7002D5B9F1000F01D022
:10CA5000202607E0302605E031465846641EFDF7E3
:10CA60002BFD0CB1A742F7D35FF00106B9F1010F1E
:10CA700002D9A9F1010903E0B5FBF6F0404502D364
:10CA800006FB08F6F2E7DFF83C9000BFB5FBF6F0D6
:10CA900000FB165519F800105846FDF70DFDB6FBC2
:10CAA000F8F6002EF2D15FEACA7009D0002C07D048
:10CAB000A74205D220215846641EFDF7FDFCF5E78C
:10CAC000BDE8F09F12CC01000A494A788B78521CCD
:10CAD000D2B2934200D100220B78934201D10020C0
:10CAE00070470270487800EB400001EBC000001D69
:10CAF00070470000941400202DE9FC411646DDE942
:10CB00000854CDE900541F468046022200F00CF87C
:10CB1000002807D1CDE900543B461022314640465B
:10CB200000F002F8BDE8FC812DE9FC5F0026DDE99C
:10CB30000C4B994692468E4680462788354630E013
:10CB4000D8F80400002200EB8500694600680190D7
:10CB500001A864DF002830D19DF8000050451FD1A6
:10CB60000EB1002100E00221228808441118594525
:10CB700022D846B9521C90B2208009F800E02088E3
:10CB8000401C20800126218801A801EB090269468A
:10CB900064DF002811D120889DF80010084420800F
:10CBA0006D1CB8F80000A842CADC56B12088C01B32
:10CBB000401E80B2FF2802D90C20BDE8FC9F09F876
:10CBC00007000020F9E7111213140D0E0F100000DA
:10CBD0007413002094130020C01300200D000300E4
:10CBE000F1A001000E000300F1A001000F000300FE
:10CBF000F1A0010010000300F1A0010000000050AE
:10CC0000D199010003000000741400200738FDD8FA
:10CC10007047303132333435363738394142434446
:10CC20004546000000000000000000000000000079
:10CC300000000000000000000000000024CC010003
:10CC40003CCC010004000000556E6B6E6F776E20C7
:10CC50006572726F7220636F6465000000000000EF
:10CC600054D201000100000000D1010002000000C8
:10CC7000F4CE01000300000074D1010004000000A4
:10CC8000C8D1010005000000A8D001000600000086
:10CC900044D0010007000000B0D1010008000000EE
:10CCA000BCD001000900000020D101000A000000F2
:10CCB0003CD201000B000000DCCE01000C000000A3
:10CCC000D4D001000D000000A4D201000E0000002D
:10CCD000A0D101000F000000DCD101001000000015
:10CCE00010D2010011000000B8D2010012000000B3
:10CCF0008CD201001300000028D201008000000047
:10CD00005CD001008100000098CF0100820000008B
:10CD100058CF01008300000038CF010084000000DC
:10CD200074CF01008500000080D001008600000063
:10CD300088D101009000000024D001009100000083
:10CD400018CF010092000000E8D00100008200002E
:10CD5000F0D10100018200003CD1010002820000FC
:10CD600058D1010000840000B4CF0100018400000C
:10CD700060D2010002840000FCCF010003840000A7
:10CD8000D8CF010041B4010029B4010021B4010051
:10CD9000FFFFFFFFFFFFFFFFFFFFFFFFFFFFFFFFA3
:10CDA00000000000000000000000D60107000000A5
:10CDB0000000000000000000000000000000000073
:10CDC00001000007B0CD0100C0CD01000800000047
:10CDD000E8CD0100F8CD010008000000F8CD010009
:10CDE00008CE010008000000C8D50100D0D5010020
:10CDF0000000000000000000B8D50100C8D5010007
:10CE00000000000000000000000000000000000022
:10CE10000000000000000000000000000000000012
:10CE200000000000000000001012002008CE0100E9
:10CE300028CE010008000000B0D50100B8D50100DF
:10CE4000000000000000000038CE010048CE0100C4
:10CE50000800000000404040404040404040414108
:10CE600041414140404040404040404040404040BF
:10CE70004040404040050202020202020202020259
:10CE80000202020202202020202020202020200256
:10CE900002020202020290909090909010101010E6
:10CEA0001010101010101010101010101010101082
:10CEB0000202020202028888888888880808080816
:10CEC00008080808080808080808080808080808E2
:10CED000020202024000000055CE01004E52465FA1
:10CEE0004552524F525F494E56414C49445F44416E
:10CEF000544100004E52465F4552524F525F534FCD
:10CF000046544445564943455F4E4F545F454E4154
:10CF1000424C4544000000004E52465F4552524F7D
:10CF2000525F464541545552455F4E4F545F454E02
:10CF300041424C45440000004E52465F4552524F1C
:10CF4000525F4D555445585F554E4C4F434B5F46CD
:10CF500041494C45440000004E52465F4552524FF5
:10CF6000525F4D555445585F4C4F434B5F464149C6
:10CF70004C4544004E52465F4552524F525F4D550C
:10CF80005445585F434F4E445F494E49545F4641B4
:10CF9000494C4544000000004E52465F4552524FF6
:10CFA000525F4D555445585F494E49545F4641497B
:10CFB0004C4544004E52465F4552524F525F424CE0
:10CFC000455F495053505F52585F504B545F545225
:10CFD000554E4341544544004E52465F4552524FD0
:10CFE000525F424C455F495053505F504545525F38
:10CFF00052454A4543544544000000004E52465FA6
:10D000004552524F525F424C455F495053505F4C1E
:10D01000494E4B5F444953434F4E4E45435445445C
:10D02000000000004E52465F4552524F525F415041
:10D03000495F4E4F545F494D504C454D454E544508
:10D04000440000004E52465F4552524F525F4E4FD1
:10D05000545F535550504F52544544004E52465F12
:10D060004552524F525F4D4F44554C455F4E4F54C1
:10D070005F494E495449414C495A4544000000001B
:10D080004E52465F4552524F525F4D4F44554C45AC
:10D090005F414C52454144595F494E495449414CC6
:10D0A000495A4544000000004E52465F4552524FD7
:10D0B000525F4E4F545F464F554E44004E52465FAE
:10D0C0004552524F525F494E56414C49445F53546A
:10D0D000415445004E52465F4552524F525F4441C3
:10D0E00054415F53495A45004E52465F4552524F94
:10D0F000525F494F5F50454E44494E470000000083
:10D100004E52465F4552524F525F5356435F48411D
:10D110004E444C45525F4D495353494E4700000021
:10D120004E52465F4552524F525F494E56414C490E
:10D13000445F4C454E475448000000004E52465F45
:10D140004552524F525F4452565F5457495F4552C1
:10D15000525F414E41434B004E52465F4552524F43
:10D16000525F4452565F5457495F4552525F444E96
:10D1700041434B004E52465F4552524F525F494E1B
:10D180005445524E414C00004E52465F4552524F5C
:10D19000525F53544F524147455F46554C4C000037
:10D1A0004E52465F4552524F525F4E554C4C000016
:10D1B0004E52465F4552524F525F494E56414C497E
:10D1C000445F504152414D004E52465F4552524FCE
:10D1D000525F4E4F5F4D454D000000004E52465F7E
:10D1E0004552524F525F464F5242494444454E00C9
:10D1F0004E52465F4552524F525F4452565F54570B
:10D20000495F4552525F4F56455252554E000000FD
:10D210004E52465F4552524F525F494E56414C491D
:10D22000445F4144445200004E52465F4552524FC3
:10D23000525F5245534F5552434553004E52465F3D
:10D240004552524F525F494E56414C49445F464CFD
:10D25000414753004E52465F535543434553530095
:10D260004E52465F4552524F525F424C455F4950C5
:10D2700053505F4348414E4E454C5F414C524541EF
:10D2800044595F4558495354530000004E52465F7D
:10D290004552524F525F434F4E4E5F434F554E548F
:10D2A000000000004E52465F4552524F525F5449B3
:10D2B0004D454F55540000004E52465F4552524F67
:10D2C000525F4255535900007761726E696E670074
:10D2D00064656275670000001B5B313B33306D0095
:10D2E0001B5B306D000000001B5B313B33316D0078
:10D2F0001B5B313B33326D001B5B313B33336D00C5
:10D300001B5B313B33346D001B5B313B33356D00B0
:10D310001B5B313B33366D001B5B313B33376D009C
:10D32000696E666F000000006572726F7200000027
:10D3300073645F626C655F6366675F7365742829F9
:10D340002072657475726E65642025732077686538
:10D350006E20617474656D7074696E6720746F20DF
:10D3600073657420424C455F47415454535F4346B4
:10D37000475F534552564943455F4348414E4745F1
:10D38000442E000073645F626C655F6366675F7361
:10D39000657428292072657475726E656420257322
:10D3A000207768656E20617474656D7074696E674E
:10D3B00020746F2073657420424C455F434F4D4D80
:10D3C0004F4E5F4346475F56535F555549442E00C5
:10D3D00073645F626C655F6366675F736574282959
:10D3E0002072657475726E65642025732077686598
:10D3F0006E20617474656D7074696E6720746F203F
:10D4000073657420424C455F47415454535F434613
:10D41000475F415454525F5441425F53495A452E2D
:10D420000000000073645F626C655F6366675F7332
:10D43000657428292072657475726E656420257381
:10D44000207768656E20617474656D7074696E67AD
:10D4500020746F2073657420424C455F434F4E4EDD
:10D460005F4346475F4741502E00000073645F6290
:10D470006C655F6366675F736574282920726574E5
:10D4800075726E6564202573207768656E206174FF
:10D4900074656D7074696E6720746F207365742095
:10D4A000424C455F4741505F4346475F524F4C45B2
:10D4B0005F434F554E542E00636C6F636B0000004A
:10D4C000434C4F434B0000004750494F5445000028
:10D4D0005052530055415254450000007077725F1E
:10D4E0006D676D740000000062616C6C6F632E6C80
:10D4F0006F675F6D656D706F6F6C000061707000BD
:10D500006E72665F736468006E72665F7364685FF4
:10D51000626C65006E72665F7364685F736F630050
:10D52000D0D50100101200202C0100004094010011
:10D530002CD601003C130020A40F0000F09901003C
:10D54000B8D4010000000000C0D4010000000000B9
:10D55000C8D4010000000000D0D401000000000089
:10D56000D4D4010000000000DCD401000000000061
:10D57000E8D4010000000003FCD401000000030314
:10D5800000D501000000030308D5010000000303DB
:10D5900014D5010000000303C0120020B8120020BF
:10D5A000C0120020F81500202813002018000000E9
:10D5B000BDC501000000000051BC010000000000DA
:10D5C0006DBD0100000000005DC40100000000000E
:10D5D00032FF135413B3201F00186A0215011223DF
:10D5E0003445566778899AABBCCDDEEFF001020373
:10D5F00004C312204240042584CD011428D3011411
:10D60000C8D2011A20081AD0081AE0041AD8041A3D
:10D61000E8041AF0041AF80411191C1A08041A1064
:0CD62000041A180451042C90D0030000E0
:040000050001920163
:00000001FF
